:020000040000FA
:100000000004040000000000A0160000A01600007C
:10001000A0160000A0160000A0160000A016000008
:10002000A0160000A0160000A0160000A0160000F8
:10003000A0160000A0160000A0160000A0160000E8
:10004000A0160000A0160000A0160000A0160000D8
:10005000A0160000A0160000A0160000A0160000C8
:10006000A0160000A0160000A0160000A0160000B8
:10007000A0160000A0160000A0160000A0160000A8
:10008000A0160000A0160000A0160000A016000098
:10009000A0160000A0160000A0160000A016000088
:1000A000A0160000A0160000A0160000A016000078
:1000B000A0160000A0160000A0160000A016000068
:1000C000A0160000A0160000A0160000A016000058
:1000D000A0160000A0160000A0160000A016000048
:1000E000A0160000A0160000A0160000A016000038
:1000F000A0160000A0160000A0160000A016000028
:10010000A0160000A0160000A0160000A016000017
:10011000A0160000A0160000A0160000A016000007
:10012000A0160000A0160000A0160000A0160000F7
:10013000A0160000A0160000A0160000A0160000E7
:10014000A0160000A0160000A0160000A0160000D7
:10015000A0160000A0160000A0160000A0160000C7
:10016000A0160000A0160000A0160000A0160000B7
:10017000A0160000A0160000A0160000A0160000A7
:10018000A0160000A0160000A0160000A016000097
:10019000A0160000A0160000A0160000A016000087
:1001A000A0160000A0160000A0160000A016000077
:1001B000A0160000A0160000A0160000A016000067
:1001C000A0160000A0160000A0160000A016000057
:1001D000A0160000A0160000A0160000A016000047
:1001E000A0160000A0160000A0160000A016000037
:1001F000A0160000A0160000A0160000A016000027
:10020000FFFFFF00FFFFFF00A0160000A016000088
:10021000A0160000A0160000A0160000A016000006
:10022000A0160000A0160000A0160000A0160000F6
:10023000A0160000A0160000A0160000A0160000E6
:10024000A0160000A0160000A0160000A0160000D6
:100800002F002200007F240000018800000000006B
:100810000C000700C0622100010020001100070049
:10082000000020000000E000020032000000020092
:10083000000000007C150200000000000040DA000B
:100840000000FE004440A900C00520000000E000B8
:100850000300320000002000A00188004440A800EE
:100860000000060091018800800078000000EB0085
:1008700015003700E280400032A0B4009101BA00B8
:10088000E280400032A0B4009102BA00E280400051
:1008900032A0B4000002EB00472BDE00F507B200E7
:1008A000602CE10004003A000059EB008301E900EC
:1008B000FDFF3E00040037006128E1000100320026
:1008C0000082EB00040007001101BA000200E00002
:1008D000E8FF3A00000006003159BA008301E90040
:1008E0000C0032002159BA008301E90008003200EF
:1008F0000400E00003003A00E280400032A0B400AF
:10090000F5FF370011D9BA008301E900FAFF3A0078
:100910008100E800E180400032A0B4000000060041
:100920007C0F0400000000006410040000000000C0
:10093000A01004000000000094100400000000005B
:100940001C0E040000000000380E0400000000002F
:100950008001EB000200370061F079008301E800BC
:10096000828F5100FCFF3A000000060012010000D7
:10097000100100000200000000080000D804000080
:100980000A00000002000000010200000301000054
:100990000902000043000000020100000080000086
:1009A00064090000040000000001000002020000D1
:1009B00001000000052400000010000001040000F8
:1009C00024020000020500002406000000010000CF
:1009D000052400000101000001070000058100005E
:1009E000030A0000004000000904000001000000AC
:1009F000020A0000000000000007000005020000DD
:100A000002400000004000000705000082020000D4
:100A100040000000400000004E4F0000454D000027
:100A2000530000000A00FA00100798002107980000
:100A300032079800430798001E009000005E88006F
:100A40002E009000105E88003E009000205E88001E
:100A50004E009000305E88000000EB00B02488005B
:100A60009424A8009424A9009EC0A9000000EB00D3
:100A700060248800F00F200070248800F00F200010
:100A8000502488000000EB00302588000000EB00B7
:100A900040258800008020004800DE00C024880037
:100AA00000082000302488008804A8000000EB0023
:100AB000405E88000000EB00505E88000000EB0004
:100AC000605E88000000EB00000F78000E00370029
:100AD0001E0078004200DD008080E800E0BC2000BD
:100AE000808040000000EB00800878001E00780045
:100AF000C200DD00E0BC2000808040000000EB0070
:100B0000800878001E0FE8001E007800EF0F5000EC
:100B1000EFFF36008000EB000000EB00F103070060
:100B20008000EB000000EB00F9030700D00020007C
:100B3000502588000000EB00706088000040EB004A
:100B400012ECB7000000EB00806088000040EB0072
:100B500013ECB70080C0B30000E8B700808120002C
:100B60001040880080C8B30001E8B7000040EB00E7
:100B700004E8B700008220003040880000C4B300C1
:100B800005E8B7000080FA00000006000000FA0047
:100B9000010037009404A80094C4BF0061406000C5
:100BA0000004E000FBFF320094C4BF000044B20028
:100BB0000004E000FCFF3A00CD42A9000080FA00EA
:100BC000000006000000FA008AC4BF006140600017
:100BD0000004E0000400320036000700100020008E
:100BE000502488002C0037008AC4BF006240600097
:100BF0000004E0000400320029000700200020006B
:100C000050248800240037008AC4BF000042B2008C
:100C10000004E0000300320000022000502488009D
:100C20001D0037008AC4BF00704060000004E0006F
:100C30000300320000012000502488001600370015
:100C40008AC4BF0001C8B300014060000004E00096
:100C50000300320000082000502488000E003700F6
:100C60008AC4BF00644060000004E0000600320057
:100C70004000200050248800070037006F00070064
:100C800080002000502488008AC4BF0068406000B3
:100C90000004E000F9FF3A000080FA0000000600BE
:100CA0000000FA00F00F2000702488000080FA0095
:100CB000000006000200FA00CDC2BF0061406000E3
:100CC00080407800CDC2BF006140600000C0680075
:100CD0006140600061416000D12C200091407800AB
:100CE000E0CFB30000C0600002407000CDE2B7006A
:100CF0000000EB0070608800800020005024880015
:100D00000000EB00806088000040EB0012ECB700B0
:100D10000040EB0013ECB7008AC4BF0068406000DD
:100D20000004E000F4FF3A000000EB0050258800CA
:100D30000000EB00602588000000EB0070258800B3
:100D40000000EB00802588000000EB009025880063
:100D50000000EB00A02588000000EB00B025880013
:100D60000000EB00C02588000000EB00D0258800C3
:100D70000000EB00E02588000000EB00F025880073
:100D80000000EB00002688000000EB001026880021
:100D90000000EB00202688000000EB0030268800D1
:100DA0000000EB00402688000000EB00B024880023
:100DB000F00F200050248800F00F200070248800DD
:100DC0000000EB00000F7800080037001E007800DC
:100DD000C200DD0000802000808040000040EB0069
:100DE000904098001E007800640F40001E007800BC
:100DF000E50F5000F5FF3600D00020005025880098
:100E000080C0B30000E8B700808120001040880057
:100E100080C8B30001E8B7000040EB0004E8B70069
:100E2000008220003040880000C4B30005E8B7000D
:100E300094A4A9000080FA00000006000200FA0055
:100E4000CDC2BF000080FB004200DE0061406000B8
:100E500080407800CDC2BF000080FB004200DE0071
:100E60006140600000C06800614060006140600057
:100E70004201DD00D12C200091407800B0CFB300BA
:100E800000C0600002407000CDE2B70090248000F6
:100E9000BAEBB700BACBBF000080FB004300DE0016
:100EA0000080FB004200DD00800078000080200010
:100EB00000804000E05D8800BACBBF000034A00095
:100EC0000080FB004300DE000080FB004200DD00EC
:100ED000800078000080200000804000F05D8800E5
:100EE000E05D8000104090008080FB00C003200087
:100EF00080806000010F7800400220009E00780092
:100F0000808F50000C003200400320009E007800CB
:100F1000808F5000040032001E007800E40F500063
:100F20000300320005003700060007000300370009
:100F3000C002070001003700A60207000080FA0087
:100F4000000006000800FA00F15D800080C0B300D8
:100F500090409800E05D8000100090001040780004
:100F60008080FB0000062000808060003107980030
:100F700000022000BE009000808F5000230032004D
:100F800000042000BE009000808F50002500320039
:100F90003E0090000000E000010032002700370012
:100FA000E05D800010009000104078000080FB00A1
:100FB0006300600020079800AE009000E18F5000B1
:100FC0000A0032002E009000E20F50000A003200AA
:100FD000AE0090000100E00001003200090037007F
:100FE000E05D80003700070015003700E05D8000FD
:100FF0007001070012003700E05D8000B1010700BA
:101000000F003700FD0207000D003700505E800022
:101010000000E0000A003200505E80000000010085
:1010200007003700605E80000000E000040032002E
:10103000505E80000000010001003700EF02070051
:10104000E15D800080C0B30080487800E05D8000F2
:1010500010079800E05D80001000900010407800BC
:101060000004E0000F003500E05D800010009000FB
:1010700066004000104078000004E00006003A00DE
:10108000E05D800010009000670040001040780094
:101090000004E0000300320081CCB300014F78006F
:1010A0000200370080C8B300004F78001E4078006F
:1010B0009E0090009040980094A4A9000080FA003F
:1010C000000006000A00FA00200798002E00900099
:1010D00090009000110798001E0090000000E800AA
:1010E000104078000080FB00400798004E00900000
:1010F000E50F500042003200CE009000E58F500016
:101100000A003C004E009000E10F50001F0032002A
:10111000CE009000E38F50002B0032004E00900074
:101120000000E0000B0032001F013700CE009000ED
:10113000E88F5000FB0032004E009000E90F500095
:1011400000013200CE009000E68F500043003200D4
:1011500015013700F05D8000900090007060800005
:1011600080487800F05D8000100090008000E8006A
:10117000706080004800DE0080487800F05D8000EC
:10118000210020008F020700080137001E00900098
:101190000080E80010407800E14F500008003A005D
:1011A00071608000D0FF2F000080600070608800B8
:1011B000F05D80008000EB0082020700FB0037003A
:1011C0008E020700F90037001E0090000080E80042
:1011D00010407800E14F500007003A007060800036
:1011E0000010A00070608800F05D80008000EB00BF
:1011F00074020700ED00370080020700EB003700A3
:101200001E00900063004000104078000004E000E1
:1012100010003A001E0090000080E80010407800A6
:101220000004E0000B0035001E0090000080E80084
:101230001040780013ECB700F05D80008000EB00F8
:1012400060020700C1E120000000EB00250207005A
:10125000D600370069020700D40037001E00900056
:1012600063004000104078000080FB0030079800C9
:101270003E009000E20F50001F003200BE009000C0
:10128000E38F50006F0032003E009000E10F5000ED
:10129000010032009D003700005E8000A0608800E1
:1012A000005E8000104078000080FB00B060880085
:1012B0001E00900067004000104078000004E0002D
:1012C00093003A001E0090006600400090407800B5
:1012D000A06080001040780080CF50008C0031006A
:1012E0001E00900066004000104078000080FB0067
:1012F000B0608800860037001E0090000080E80083
:1013000090407800005E800071004000104078003E
:1013100080CF50000100390038020700105E8000C5
:10132000A0608800A06080000080E8001040780085
:101330008080FB00A06080006300400010407800C7
:101340000080FB004800DD0000804000B0608800A5
:101350000000EB00000F780010003700A160800053
:10136000B060800000804000A0608800A060800025
:101370000080E800104078008080FB00A0608000C2
:1013800063004000104078000080FB004800DD0052
:1013900000804000B06088001E0FE8001E00900032
:1013A0000080E800104078000080FB009E0F500095
:1013B000EAFF3C001E00900067004000904078006B
:1013C000A0608000630040001040780080CF500093
:1013D000100039001E009000670040009040780027
:1013E000A0608000630040001040780080CF500073
:1013F00047003A001E0090006600400090407800D0
:10140000A06080000080E8001040780080CF50008D
:101410003F0031001E009000660040001040780040
:101420008080FB001E0090006700400010407800A4
:101430000080FB004800DD0000804000B0608800B4
:10144000330037001E0090000080E8001040780054
:101450008080FB00305E8000808F500001003500EE
:10146000E6010700205E8000A0608800A060800088
:10147000104078000080FB00B06088000000EB00A6
:10148000000F780009003700A1608000B060800084
:1014900000804000A0608800A060800010407800BC
:1014A0000080FB00B06088001E0FE8001E00900066
:1014B0000080E800104078000080FB009E0F500084
:1014C000F1FF3C001E0090006700400010407800D3
:1014D0000004E0000E003A001E009000660040008C
:1014E00090407800A06080001040780080CF5000CD
:1014F000070031001E009000660040001040780098
:101500000080FB00B060880001003700BB010700CD
:10151000D701070081E320000000EB007101070004
:1015200022003700F05D8000900090008060800015
:1015300080487800F05D800011002000A1010700C4
:101540001A0037001E0090000080E800104078006C
:10155000E14F500012003E001E0090000080E800A5
:10156000104078000080FB00806088008060800070
:101570000000E0000400320000C2B30012ECB7002B
:10158000350207000200370000C1B30012ECB700BB
:10159000F05D80008000EB008A0107000300370047
:1015A0009601070001003700940107000080FA004F
:1015B000000006000600FA00100798001E009000C8
:1015C00090009000010F78001E00E80010407800A5
:1015D0000080FB00200798002E0090000000E00033
:1015E0000A003200AE0090000100E0003200350039
:1015F0002E009000EA0F500011003200AE00900063
:10160000EB8F50001D0032002B003700F05D800092
:10161000900090000040EB0080487800F05D800072
:10162000100090008000E8000040EB008048780047
:10163000F05D800021002000620107001F003700DC
:101640009E0078006480400010407800E14F500018
:1016500008003E00F05D8000900090000040EB002C
:1016600080487800F05D80001100200055010700DF
:101670001200370061010700100037009E0078005B
:101680006480400010407800E14F500008003E00A8
:101690001E80E800104078000004E00004003A00DA
:1016A000F05D80008000EB0046010700030037007A
:1016B0005201070001003700500107000080FA00C6
:1016C000000006000A00FA00300798003E00900073
:1016D00090009000210798002E0090000000E80084
:1016E000104078000080FB00400798004E009000FA
:1016F000E10F500051003200CE009000E38F500007
:10170000800032004E0090000000E0000100320036
:10171000AD003700F05D8000900090000040EB00CD
:1017200080487800F05D8000100090008000E800A4
:101730000040EB00804878002E00900064004000DC
:10174000104078006F406000304798002E009000F5
:1017500064004000104078000080FB004700DE007D
:10176000204798003E4090000080FB0000004000B1
:10177000800078002E4090000080FB000080400038
:101780004200DD008000780000802000008F4000D3
:101790001E00780090409000B0CFB30080C0600081
:1017A0001E007800114098001E0078001040900044
:1017B0000004E00004003200F05D80009000900022
:1017C00010C0B300804878003E4090000080FB00CD
:1017D00000004000800078002E4090000080FB0058
:1017E000008040004200DD00800078000080200082
:1017F000008F40001E00780090409000B0CFB300F2
:1018000080C060001E007800114098001E00780023
:10181000104090000004E00004003200F05D800001
:101820009000900010C0B30080487800F05D800008
:1018300021002000E3000700640037002E00900024
:1018400064004000104078006F406000304798000E
:101850002E00900064004000104078000080FB00E3
:101860004700DE00204798003E4090000080FB00CB
:1018700000004000800078002E4090000080FB00B7
:10188000008040004200DD008000780000802000E1
:10189000008F40001E00780090409000B0CFB30051
:1018A00080C060001E007800114098002E4090001B
:1018B0000004E000060032001E0078009040900016
:1018C00000C4B30080C070001E0078001140980072
:1018D0002E4090000004E00006003A001E00780050
:1018E00090409000F0CBB30080C060001E007800F4
:1018F00011409800F05D80008000EB00B10007000F
:10190000320037002E009000640040001040780044
:101910006F406000304798002E0090006400400047
:10192000104078000080FB004700DE002047980050
:101930003E4090000080FB000000400080007800E6
:101940002E4090000080FB00008040004200DD003F
:101950008000780000802000008F40001E0078008A
:1019600010409000804078000124A0001E00780004
:10197000114098003E4090000080FB0000004000B5
:10198000800078002E4090000080FB000080400026
:101990004200DD008000780000802000008F4000C1
:1019A0001E00780010409000804078000124A000C4
:1019B0001E00780011409800F05D80008000EB0070
:1019C00080000700010037008C0007000080FA004B
:1019D000000006000000FA00BACBBF000080FB0048
:1019E0004400DE000080FB006F006000C200DD00EC
:1019F000E0BC200000804000100078000000E00003
:101A00000A003200BACBBF000080FB004400DE00B9
:101A10000080FB006F006000C200DD00E0BC200021
:101A20000080400010007800000001000080FA00F3
:101A3000000006000000FA00BACBBF000080FB00E7
:101A40004400DE000080FB006F0060004200DD000B
:101A50008080E800E0BC200000804000100078009A
:101A60000000E0000B003200BACBBF000080FB009A
:101A70004400DE000080FB006F0060004200DD00DB
:101A80008080E800E0BC200000804000100078006A
:101A9000000001000080FA00000006000200FA00C9
:101AA000000F78001E007800405E88000080FA0079
:101AB000000006000200FA00000F78001E00780007
:101AC000505E88000080FA00000006000200FA0064
:101AD000000F78001E007800605E88000080FA0029
:101AE000000006000400FA00000F780011079800BB
:101AF0001E007800C200DD00E0BC20000080400035
:101B00009E009000010878000080FA0000000600A6
:101B10000400FA00000F7800110798001E007800FA
:101B20004200DD008080E800E0BC20000080400032
:101B30009E009000010878000080FA000000060076
:101B40000200FA00000F78001E007800904090001C
:101B500000C4B30000C0680002C4B300824060004B
:101B600080C8B30000C07000804078001E0078007C
:101B7000114098000080FA00000006000200FA0000
:101B8000000F78009E0078000040EB00804878004D
:101B90001E0078009040900000C4B30000C06800B0
:101BA00002C4B3008240600080C8B30000C070006F
:101BB000804078001E007800114098000080FA00F4
:101BC000000006000400FA00000F780011079800DA
:101BD0001E0090008040780000C0EB0080C06000D4
:101BE0001E007800014878009E00780080CCB30089
:101BF000904098000080FA00000006000000FA0003
:101C000080C0B30000E8B70080C0B30000E8B700B0
:101C100040C8B30005E8B70040C8B30001E8B7000A
:101C200040C8B30005E8B70040C8B30001E8B700FA
:101C30000080FA00000006000000FA0013CCBF008C
:101C40000004E0000500350013CCBF000080FB005D
:101C5000B024880000C0EB0013ECB7008000EB005C
:101C60000000EB009FFF07000080FA000000060064
:101C70000600FA00B06080000000E0001C003200A6
:101C8000B0608000200798002E009000E80F500000
:101C90000200360083002000230798002E009000E9
:101CA000000F78000000EB00100798000C003700D0
:101CB000F05D8000900090001E00900000814000C8
:101CC000A16080001E00900000804000104078005D
:101CD000004978001E0090000000E80010079800FE
:101CE0001E0090009E0F5000F1FF390005003700E4
:101CF0000000EB00000F78008000EB000000EB001C
:101D000078FF0700F15D80001E00780080487800B1
:101D1000F25D8000F05D80009040900000C4B30050
:101D200000C0680003C4B3008340600080C8B300F3
:101D300000C0700010419800A16080001E00780073
:101D400000804000A0608800B06080001E0050004D
:101D5000B06088000080FA00000006000200FA006F
:101D60008EC0BF000044B2000004E000200032003A
:101D70008AC4BF00614060000004E0000600320039
:101D8000CCFB07001000200050248800F00F20003A
:101D9000000F7800180037008AC4BF006840600058
:101DA0000004E0001100320090248000BAEBB7007C
:101DB000BACBBF000080FB004400DE000080FB00C7
:101DC0006F0060000000E000060032001BFC07000E
:101DD0008000200050248800F00F2000000F7800C1
:101DE0000500370080002000502488008EC0A90024
:101DF0000000EB00000F78001E0078000080FA0061
:101E0000000006000000FA0000202C001100200055
:101E1000D05C8800E15C88000000EB00F05C88008A
:101E20000000EB00005D880080C0B300A2EBB700AB
:101E3000A40BA900A42BA900C0F720001DFF0700D8
:101E40000000EB00905D8800905D8000805D880060
:101E50000080FA00000006000000FA008000EB009D
:101E6000100020001FFF07008000EB002000200072
:101E70001CFF07008000EB002000200024FF07006B
:101E80005001200060258800D001200070258800C6
:101E90000040EB000CE8B700E0B420007040880080
:101EA00080C4B3000DE8B70000C4B30010E8B70069
:101EB000E0AC20009040880080C8B30011E8B70073
:101EC0000040EB0014E8B700E0B02000B04088000C
:101ED00080C4B30015E8B700C0F72000F5FE070086
:101EE00000812000A05D880040812000B05D880056
:101EF0000080FA00000006000600FA00CDC2BF0014
:101F00000080FB000000D10061406000804078004C
:101F1000CDC2BF000080FB000000D1006140600026
:101F200000C0680061406000614060000041400006
:101F3000D12C200091407800D0CFB30000C06000C9
:101F400002407000CDE2B700E05D8000900090009C
:101F5000110798001E009000104078008080FB0060
:101F6000300620008080600010022000808F50002A
:101F7000010032004B0037001E0090000000E80016
:101F8000104078000080FB00200798002E00900091
:101F9000E40F50000A003C00AE009000E28F5000B9
:101FA0001C003D002E0090000000E00011003200F7
:101FB000AE009000E18F5000120032003700370071
:101FC00010022000AE009000808F500017003200F9
:101FD00020022000AE009000808F500024003200CC
:101FE00000022000AE009000808F50000B003200F5
:101FF0002A003700F05D80008000EB00F1FE070052
:1020000029003700F05D80008000EB00EDFE070046
:1020100025003700F9FE07002300370041062100A4
:102020000000EB00BAFE07001F0037001E00900002
:1020300066004000100F7800A00020009E0F1000E6
:1020400002003600A0002000000F7800F05D800044
:1020500010009000A1B920001E0178003CFA070092
:102060009E007800F05D8000D6FE07000E0037006D
:102070001E0090000080E80010007800205D8800BD
:10208000010A21000000EB0096FE0700F05D8000D1
:102090008000EB00CBFE070003003700D7FE0700EF
:1020A00001003700D5FE07000080FA00000006009E
:1020B0000000FA008000EB000000EB0089FE070042
:1020C0000080FA00000006000000FA00E05D8000D9
:1020D00010009000A1B9200009000900B058780054
:1020E000A000B1008000EB000000EB0088FE0700BC
:1020F000410921000000EB007AFE0700F05D80003E
:102100008000EB00AFFE0700E15D800080C0B300FF
:1021100080487800E15D800080C8B300904098005E
:102120000080FA00000006000000FA008000EB00CA
:102130000000EB006BFE07000080FA0000000600C4
:102140000000FA008000EB000000EB0065FE0700D5
:102150000080FA00000006000000FA00C05D800068
:102160000000E00003003200C05D80000000E900D4
:10217000C05D88000080FA00000006000200FA003E
:102180000A0037009EC0BF000044B2000004E00017
:1021900006003A00F1FE07000004E00003003200F0
:1021A0000000EB00000F780006003700A05D800003
:1021B000104090000004E000F2FF35001000200005
:1021C000000F78001E0078000080FA000000060072
:1021D0000200FA000A0037009EC0BF000044B200AF
:1021E0000004E00006003A00DCFE07000004E00006
:1021F000030032000000EB00000F780006003700FB
:10220000B05D8000104090000004E000F2FF350057
:1022100010002000000F78001E0078000080FA00F7
:10222000000006000600FA00000F78002147980021
:102230000A0037009EC0BF000044B2000004E00066
:1022400006003A00C5FE07000004E000030032006B
:10225000F00F20002007980018003700B05D8000C4
:10226000104090000004E000F2FF3500B05D8000F7
:102270009E00780011009800B05D8000AE41900093
:1022800003487800B25D8000B05D8000904090000F
:1022900000C4B30000C0680003C4B3008340600002
:1022A00080C8B30000C0700010419800ABFE07006A
:1022B0002E4090000080FB00200798002E00900028
:1022C0000080FA00000006000200FA00A05D800015
:1022D000104090008000EB00010F78000004E00047
:1022E0000200350010002000000F78001E0078006A
:1022F0000080FA00000006000200FA00B05D8000D5
:10230000104090008000EB00010F78000004E00016
:102310000200350010002000000F78001E00780039
:102320000080FA00000006000400FA00000F7800A8
:10233000214798000040EB00A7EBB700A05D8000AC
:10234000104090000004E0002E003500A05D8000E9
:10235000904078002E40900080CF50000300310064
:10236000A05D800090407800214798000040EB007D
:10237000A7EBB7000C003700A7CBBF000080FB0025
:102380001E014000A7CBBF008080FB00E0AC200016
:10239000008040001040780000497800A7CBBF00C3
:1023A0000040E800A7EBB70071BA20009140780028
:1023B0002E40900080CF5000EFFF39009EC0BF003C
:1023C0000044B2000004E00001003A0063FE070090
:1023D000A15D800000C4B30080487800A25D800049
:1023E000A05D80009040900000C4B30000C0680071
:1023F00003C4B3008340600080C8B30000C0700015
:1024000010419800A7CBBF000080FB000080FA00BD
:10241000000006000000FA0098CBBF000004E000B6
:1024200007003A0001C4B30080B52000BEFF0700DA
:1024300098EBB700E3F907000040EB0099EBB70019
:102440000080FA00000006000200FA00000F780089
:10245000F0FF070098CBBF000004E000FCFF320053
:1024600099CBBF008080FB0080B520000080400039
:10247000904078001E0078000148780098CBBF009B
:102480000040E90098EBB70099CBBF000040E8009E
:1024900099EBB700100020000080FA000000060051
:1024A0000800FA000040EB0006EAB7000000370021
:1024B000C4F90700D7FF070000A02000E2FF0700D3
:1024C0000004E000FAFF320001A0200091407800F3
:1024D00010CCB30080CF5000F5FF3A003CFF07005E
:1024E00010CFB3000EEBB70040C0B3000FEBB70046
:1024F00060C0B30010EBB70031C0B300E0B0200003
:1025000048FF0700B0C4B30007EAB7000000370077
:10251000ACF907002EFF070007CABF000EEBB7009B
:1025200011C0B300E0B020003EFF07000040EB0008
:10253000004F780080A02000C3FF070008CABF003A
:102540001E4F400090A02000BFFF070009CABF0037
:102550001E4F4000A0A02000BBFF07000ACABF001A
:102560001E4F4000B0A02000B7FF07000BCABF00FD
:102570001E4F4000C0A02000B3FF07000CCABF00E0
:102580001E4F400008CABF000080FB009001880079
:102590000CCABF00E14F5000180036000000EB00ED
:1025A000100798000E0037001E0090008000780091
:1025B000E0A0200000804000A3FF07001E00900064
:1025C000E800400060A0200000804000104078003B
:1025D0001E4F40001E0090000000E8001007980009
:1025E0000CCABF000080FB000000E90080007800FA
:1025F0001E009000808F5000EBFF3E00D0A0200016
:1026000091FF07000DCABF001E4F40001E04E000EE
:1026100003003200E0C4B30007EAB700BCFF370094
:1026200008CABF000080FB00010020001050880095
:10263000215088001050800021508000C808DD0023
:102640000080FD00804078000040EB0010508800C2
:102650002150880009CABF000081FB000300200050
:10266000105080002150800002004000838048000C
:1026700010508800215088001050800021508000A8
:10268000C808DD000080FD00804078000040EB00BD
:1026900010508800215088000ACABF000081FB004A
:1026A00003002000105080002150800002004000F4
:1026B0008380480010508800215088000BCABF005A
:1026C0000080FB00300798003E009000E20F5000B1
:1026D0000B003200F00F2000BE009000808F5000F1
:1026E000090032003E009000E10F5000010032006E
:1026F0001800370010C0B30006EAB7001700370013
:102700001B000700150037009404A9000080EB00AF
:1027100020079800080037000080EB0010079800A1
:102720001E0090000000E900100798001E009000B5
:10273000E10F4000FAFF3A002E0090000000E9008F
:10274000200798002E009000E10F4000F2FF3A00B1
:102750000000FE0050C5B30007EAB7006ACCBF0016
:102760000004E0006AFF32000080FA00000006006A
:102770000C00FA000040EB00004F78001050800081
:1027800021508000E00F5000E08F58000C003A000C
:1027900040C0B3000EEAB7000040EB000FEAB700FC
:1027A00040C0B30010EAB7000040EB0011EAB700E8
:1027B0000040EB0012EAB7000040EB0013EAB7005C
:1027C0001250800023508000F0FF21000100200003
:1027D000800F5100818F59000B003C001250800087
:1027E00023508000F03F200001002000800F5100A6
:1027F000818F59000400340000C5B30007EAB70018
:1028000010C0B300004F78001250800023508000A9
:10281000F07F2A0021002000800F5100818F590095
:102820000400340000C5B30007EAB70010C0B300CD
:10283000004F78001E04E000AD003A0006CABF0059
:102840000004E0001600320020042400003B880051
:102850001050800021508000800078000080EB0044
:102860008008BB004E00900050052000303B8800DF
:10287000A00A2000303B880061E7A80000000000AB
:102880000000000061C7BF0001C8B3000140600044
:102890000004E000FBFF3A000040EB0006EAB7004E
:1028A0001050800021508000100798001000240074
:1028B000003B88000040EB00604798002D00370087
:1028C0006E4090000080FB00E800400060A0200007
:1028D00000804000104078000080FB002007980036
:1028E000AE0090001E0090000188BB006E4090007A
:1028F0000040E800604798006E4090000080FB00B8
:10290000E800400060A020000080400010407800F7
:102910000080FB00200798006E4090000040E80017
:10292000604798006E4090000080FB00E800400087
:1029300060A0200000804000104078000080FB0074
:10294000C800DD002E0090000100700020079800F4
:102950006E4090000040E80060479800AE00900094
:102960001E0090000108BB001E0090000080E800DF
:10297000100798006E4090008080FB000CCABF00DA
:102980000080FB000000E900808F5000CCFF350084
:102990005E00900050052000303B8800A00A200017
:1029A000303B880061E7A800000000000000000044
:1029B00061C7BF0001C8B300014060000004E0002F
:1029C000FBFF3A0061C7A900105080002150800031
:1029D00010079800B0C4B30007EAB7000040EB004E
:1029E000604798003B0037001E0090001080BA003E
:1029F00020079800AE009000F00F200000806000DB
:102A0000200798006E4090000080FB00E800400026
:102A100060A0200000804000104078008080FB0013
:102A20002E009000808F50000200320060C5B3007D
:102A300007EAB7006E4090000040E8006047980049
:102A40001E0090001000BA00200798002E00900091
:102A5000004178006E4090000080FB00E8004000DC
:102A600060A020000080400010407800804F51009E
:102A70000200320060C5B30007EAB7006E40900064
:102A80000040E800604798002E0090004880DE007B
:102A9000004178006E4090000080FB00E80040009C
:102AA00060A020000080400010407800804F51005E
:102AB0000200320060C5B30007EAB7006E40900024
:102AC0000040E800604798001E0090000080E80089
:102AD000100798006E4090008080FB000CCABF0079
:102AE0000080FB000000E900808F5000BEFF350031
:102AF0000080FA00000006000200FA000080EB00EF
:102B000060198800C8E2A8006F20A800CCC2A90004
:102B1000C8C2A90080382100000F78001E0078008C
:102B20000000E900000F78001E007800E10F40006F
:102B3000FAFF3A000000EB00000F78000A003700AF
:102B4000CAC2BF0001C8B300014060000004E00039
:102B50000200320001002200014001001E00780046
:102B60000000E800000F78001E007800F30F50000E
:102B7000F3FF34006F20A900C8C2A80003000700BB
:102B80000000EB000080FA00000006000000FA00E0
:102B900016000700C902A900C922A900C942A9005C
:102BA000CD42A800CD02A900CD22A80043002000FC
:102BB00082C12000814C2800604B280099F7070053
:102BC000F2F707008FFC0700CD22A900FDF70700F0
:102BD00012CCBF00FF4F5000FCFF3600CD22A800F2
:102BE0002FFE07000080FA00000006000000FA0037
:102BF0004440A8000000EB00A00188000000EB00AA
:102C0000203A88000000EB00900188000080EB0073
:102C10006019880020002000501988000080EB0017
:102C2000401688000080EB00801688000080EB00D2
:102C3000C01688000080EB00001788000080EB00C1
:102C4000401788000080EB00801788004227A90009
:102C50000080FA00000006006A0C0000020000007C
:102C60000200000000000000000A0000CE0000008A
:102C70000000000000200000020000000000000032
:102C80006C0C0000020000000200000000000000C8
:102C9000580B00006200000000000000CE0A000097
:102CA0008A00000000000000180C00005200000024
:102CB0000200000004030900042A0300440061002C
:102CC000006E000067006500007200006F00750074
:102CD0000073000020005000007200006F007400BC
:102CE000006F000074007900007000006500730040
:102CF0000012030043004400004300002000540081
:102D00000065000073007400001203003000300002
:102D10000030000030003000003000003000310092
:102D20000000000000080000000200000000000099
:102D3000BA0B00005E000000000000000000000070
:102D40000000FE00FFFFFF00FFFFFF00FFFFFF008E
:102D5000FFFFFF00FFFFFF00FFFFFF00FFFFFF007F
:102D6000FFFFFF00FFFFFF00FFFFFF00FFFFFF006F
:102D7000FFFFFF00FFFFFF00FFFFFF00FFFFFF005F
:102D8000FFFFFF00FFFFFF00FFFFFF00FFFFFF004F
:103FE000FFFFFF00FFFFFF00FFFFFF0006040000D0
:103FF0000000FA00E5FA07000080FA000000060061
:10400000FFFFFF00FFFFFF00FFFFFF00FFFFFF00BC
:10401000FFFFFF00FFFFFF00FFFFFF00FFFFFF00AC
:10402000FFFFFF00FFFFFF00FFFFFF00FFFFFF009C
:10403000FFFFFF00FFFFFF00FFFFFF00FFFFFF008C
:020000040005F5
:1057F00000000000FFFF00009E2300007F3E00002D
:00000001FF
